:020000040000FA
:1000000090040020D50000005B08000059080000A3
:1000100000000000000000000000000000000000E0
:10002000000000000000000000000000C9080000FF
:1000300000000000000000009D080000CD08000046
:10004000E7000000E7000000E7000000E700000014
:10005000E7000000E7000000E7000000E700000004
:10006000E7000000E7000000E7000000E7000000F4
:10007000E70000000000000000000000E7000000B2
:10008000E700000000000000E7000000E7000000BB
:1000900000000000E700000000000000790A0000F6
:1000A000E7000000E7000000000000000000000082
:1000B000E7000000E700000000000000E70000008B
:1000C0000348854600F000F900480047150F00007E
:1000D000900400200448804704480047FEE7FEE7FC
:1000E000FEE7FEE7FEE7FEE705090000C1000000AD
:1000F00030B50B46014600202022012409E00D46C0
:10010000D5409D4205D31D469540491B2546954047
:1001100040191546521E002DF1DC30BD70B5024667
:100120004A40D50F40004A00ED0740085208002819
:1001300014D0002A12D0C40DD30D41020120C005F5
:100140005202490A520AE41A091812187D349142DF
:1001500001D3641C00E04900002C01DA002070BDCE
:100160000023914201D3891A034340084900002823
:10017000F7D100290AD0914202D10121C90705E037
:10018000914201D2012101E00121C943E005C018DB
:10019000401900F058F870BD420005D04200120E20
:1001A00052428A4201DB00207047C9050818704797
:1001B00010B500229623114600F04DF810BD410005
:1001C00040020122400AD205090E80187F2901DA77
:1001D00000207047962903DC9622511AC8407047C8
:1001E000963988407047C20FD207400040080BD0B4
:1001F000C10D0723DB01C91840020905400A11435C
:10020000C208400711437047002001467047CB0FDA
:10021000DB07490010B5490802460A4307D00A0D1A
:1002200007240903E401090B121B002A01DC00204A
:1002300010BDC900440F0C43C100E018D20580185E
:1002400000F001F810BD002904DA401C490001D17A
:1002500040084000704770B40024050C05D11024FC
:10026000000402D1002921D01124050E01D1000281
:100270000834050F01D10001241D850F01D1800034
:10028000A41C002801DB4000641C002908D02025A4
:100290002E1B0D46F540A14000D001212943084303
:1002A00001061B1B000ADB1D02D5002070BC704735
:1002B000DB05181880180029F8DA401C4900F5D130
:1002C00070BC400840007047064C0125064E05E012
:1002D000E36807CC2B430C3C98471034B442F7D367
:1002E000FFF7F2FE301600005016000001218907CA
:1002F0000868C007C00F01D0054A0A600022054BFC
:10030000D2439A60002801D00020086070470000A6
:100310009669AA554000004000B5030000F072FC49
:100320002B171945454545454527292B2D2F314587
:10033000191B1D1F21232527292B2D2F313335373D
:100340004545454545393B3D3F4541434500002036
:1003500000BD012000BD022000BD032000BD04201F
:1003600000BD052000BD062000BD072000BD0820FF
:1003700000BD092000BD0A2000BD0B2000BD0C20DF
:1003800000BD0D2000BD0E2000BD0F2000BD1020BF
:1003900000BD162000BD172000BD182000BD19208B
:1003A00000BD1B2000BD1C2000BDFF2000BD30B5DE
:1003B000054608780C4601280FD00021284600F099
:1003C000DBF9A178284600F073F86178284600F040
:1003D00059F86078002812D019E00121284600F071
:1003E000CBF90121284600F04DF80021284600F005
:1003F0005FF80021284600F077F9002110E021790C
:10040000284600F027F8E178284600F03DF9012160
:10041000284600F099F96179284600F065F9A1793C
:10042000284600F049F90021284600F075F930BD52
:1004300000B50146FFF770FF0D2901D8044901E01E
:10044000034980390968C140C807C00F00BD0000DA
:100450008004004010B50446FFF75EFF01220D2C1A
:1004600003D8074B03E0596010BD054B803B0029C2
:10047000596802D082401143F5E782409143F2E788
:10048000C004004010B50446FFF746FF01220D2CC2
:1004900007D8064B07E082409A6110BD8240DA61BE
:1004A00010BD024B803B0129F8D1F4E780040040E5
:1004B000F0B5002906D0012904D0022902D0032971
:1004C00000D0FF2130256F4A6E4C2E022F03803A58
:1004D000030000F097FB2B171D2323232323232442
:1004E0002A2F363B4023494E555A5F666D767C81F4
:1004F000888D9299A0A92323232323AFB6BFC523B8
:10050000CACF2300606A890780088000890F03E052
:10051000606A8907A843890E08436062F0BDA06A3B
:10052000890780088000890F1BE0A06A8907A8431B
:10053000890E16E0A06A0322120290438907890DF2
:100540000FE0A06A8907B043890C0AE0A06A890716
:10055000B843890B05E0A06A03221205904389077E
:10056000890A0843A062F0BD506A8907A843890E32
:1005700024E0506A03231B0298438907890D1DE07C
:10058000506A8907B043890C18E0506A8907B8435C
:10059000890B13E0506A03231B0598438907890AD6
:1005A0000CE0506A03231B0698438907890905E07C
:1005B000506A03231B079843890789080843506240
:1005C000F0BD906A890780088000890F29E0906A51
:1005D0008907A843890E24E0906A03231B029843ED
:1005E0008907890D1DE0906A8907B043890C18E0DE
:1005F000906A8907B843890B13E0906A03231B05AF
:1006000098438907890A0CE0906A03231B069843E4
:100610008907890905E0906A03231B079843890726
:10062000890808439062F0BDD06A8907800880007D
:10063000890F0CE0D06A03231B06984389078909B8
:1006400005E0D06A03231B079843890789080843FC
:10065000D062F0BD106B890780088000890F0DE023
:10066000106B8907A843890E08E0106B8907B04317
:10067000890C03E0106B8907B843890B08431063AA
:10068000F0BD00008004004010B50446FFF744FEB2
:1006900001220D2C03D8074B03E0996310BD054BD5
:1006A000803B0029996B02D082401143F5E78240DC
:1006B0009143F2E78004004010B50446FFF72CFE9A
:1006C00001220D2C03D8074B03E0196010BD054B28
:1006D000803B0029196802D082401143F5E782402F
:1006E0009143F2E7C004004010B50446FFF714FE42
:1006F00001220D2C03D8074B03E0D96310BD054B35
:10070000803B0029D96B02D082401143F5E782403B
:100710009143F2E78004004010B50446FFF7FCFD6A
:1007200001220D2C03D8074B03E0D96010BD054B07
:10073000803B0029D96802D082401143F5E782400E
:100740009143F2E7C004004010B50446FFF7E4FD12
:1007500001220D2C03D8074B03E0996010BD054B17
:10076000803B0029996802D082401143F5E782401E
:100770009143F2E7C004004010B50446FFF7CCFDFA
:1007800001220D2C03D8074B03E0596310BD054B24
:10079000803B0029596B02D082401143F5E782402B
:1007A0009143F2E78004004010B50446FFF7B4FD22
:1007B00001220D2C07D8064B07E082409A6010BD3D
:1007C0008240DA6010BD024B803B0129F8D1F4E78A
:1007D0008004004030B501241D4BA407236002258E
:1007E0001C4B012858680DD04008400058605868DC
:1007F000A8435860186880088000401C18600020DA
:10080000206030BD800309D458684008400058601B
:1008100058682843586058688003FCD5206A00094E
:100820000001401C206258680C258907A843090F65
:1008300008435860012A03D058688003FCD5DEE7DE
:10084000186880088000186058688003FCD5D6E7D7
:100850009669AA5540000040FEE7704730B5C406CF
:10086000E40E0123A340002A10D08408094AA40002
:10087000A21814688007C00EFF2585408907090E5D
:10088000AC43814021431160034801E002488030BD
:10089000036030BD00E400E000E100E070470000CC
:1008A0000121074A89070A60064A136880079B08E6
:1008B0009B00800F03431360002008607047000016
:1008C0009669AA5540000040704700000248016840
:1008D000491C01607047000084000020084A03683A
:1008E0000021536191610379002B00D004214379E9
:1008F0000220002B01D0014300E0814311617047C9
:1009000000E000E010B50020FFF7CAFF10BD02694B
:1009100006239A430B789B075B0F1A430261026917
:1009200008239A434B78DB071B0F1A4302610269C5
:1009300030239A438B789B079B0E1A43026102690E
:10094000C0239A43CB789B071B0E1A430261C268EF
:100950000979120A1202491EC9B20A43C2608169AA
:100960008022914381617047016949084900016112
:100970007047016901221143016170470269032335
:100980001B0389079A43890C0A43026170478269F5
:1009900003231B0389079A43890C0A43826170472A
:1009A000026903239B0389079A43090C0A430261E6
:1009B0007047826903239B0389079A43090C0A4302
:1009C0008261704782690B7852085200DB07DB0FA7
:1009D0001A438261826902239A434B78DB079B0F9B
:1009E0001A438261826904239A438B78DB075B0F89
:1009F0001A438261826908239A43CB78DB071B0F75
:100A00001A438261826930239A430B799B079B0EBC
:100A10001A438261826940239A434B79DB075B0E5C
:100A20001A438261826989798023C9079A43090E32
:100A30000A438261704703690122120493430361F0
:100A400043681B0C1B040B434360016911430161A4
:100A50007047826B120C12040A4382637047C26BA8
:100A6000120C12040A43C2637047426C120C120447
:100A70000A4342647047000010B5044C204600F061
:100A800089F80146204600F088F810BD006000405B
:100A9000C16170470246D26900200A4200D001209D
:100AA0007047012A826902D08A43826170470A43F3
:100AB000FBE70000F8B50D460E7B344904460020E4
:100AC0000F68012E06D0022E07D0032E08D0042E68
:100AD00009D013E0A868000107E0A868400104E01D
:100AE000A868800101E0A868C001FFF761FB0090E1
:100AF0003846FFF75DFB0099FFF710FB7F21C90522
:100B0000884202DA0020224901E0FFF76CFBFFF780
:100B10007EFB0421FFF740FBFFF751FB61680722D2
:100B2000120291437207520D1143616020612068E7
:100B30000121490388432978C907890C08432060AB
:100B400020680F210902884369780907090D0843C5
:100B500020602068012109038843A978C907C90CCE
:100B60000843206020680F2109068843E9780907B7
:100B70000909084320602068012109078843297971
:100B8000C907C90808432060F8BD000080000020A4
:100B90000000F03F2030007970472030017070472E
:100BA0004268890792089200890F0A4342607047A1
:100BB0001CB50A487D21C9000068FFF799FA00902A
:100BC00001206946087148716846FFF787FE0448AE
:100BD00001694908490001611CBD00008000002036
:100BE00000E000E00FB410B503A9044B044A0298DA
:100BF00000F024F810BC08BC04B018478D0D0000AC
:100C00008800002030B47446641E2578641CAB4212
:100C100000D21D46635D5B00E31830BC184702E05C
:100C200008C8121F08C1002AFAD170477047002077
:100C300001E001C1121F002AFBD17047FFB58DB042
:100C40000446002506E025280AD0109A0F999047FF
:100C5000641C6D1C20780028F5D1284611B0F0BD29
:100C600000270121484A009700E00743641C2378CD
:100C70000846203B98401042F7D120782E2817D103
:100C8000042007436078641C2A280CD10E98641C49
:100C900002C800910E900BE000990A2251433039AE
:100CA0004018641C00902078014630390929F3D996
:100CB00020780028D1D0642808D0692806D075286B
:100CC0001ED0109A0F9990476D1C5BE00A200E9978
:100CD000019001C90E91002802DA40422D2102E064
:100CE000390504D52B216A461172012103E0F90769
:100CF00004D02021F7E70BAE0B910DE00021FAE7BD
:100D00000A200E99019001C90E91F7E70199FFF7AA
:100D1000EFF93031761E31700028F7D103A8801B1F
:100D200020300190780701D5009801E00120009063
:100D30000199884201DD401A00E000200027009060
:100D400006E002A8109AC05D0F9990476D1C7F1CA9
:100D50000B988742F5DB04E0109A30200F999047FA
:100D60006D1C0099481E00900029F5DC05E03078E4
:100D7000109A761C0F9990476D1C0199481E01909E
:100D80000029F4DC641C65E709280100F8B50E4F62
:100D90000646C1B200243846FFF7FFFE0B4D022184
:100DA0003846FFF777FE641C002801D1AC42F6D12B
:100DB00002213846FFF76CFEAC4202D10020C0434E
:100DC000F8BD3046F8BD000000600040E21C0000A5
:100DD00070B50A48C1680A48006800F0AFFA094DCA
:100DE000002403202C6000F00FF8042000F020FB0A
:100DF000EC6000206C6000F08FF970BD5C0000209A
:100E0000580000206C00002010B500280AD00128EE
:100E10000AD0022810D0032817D1002000F0D8F9FA
:100E2000002005E00120F9E7002000F0D1F90120C1
:100E300000F0C7F9002006E0002000F0C9F900200A
:100E400000F0BFF9012000F0B5F910BD01480068BD
:100E500070470000840000201CB500F02FF800202F
:100E60006A461070012151709070507191716946FD
:100E70001920FFF79CFA69461E20FFF798FA694689
:100E80001B20FFF794FA1CBD10B5084CA06800F0B9
:100E900059F92169884207D3FFF7D8FFA060FFF70F
:100EA00097FF03A0FFF79EFE10BD00006C0000201E
:100EB00074696D65206F7665720D0A001CB500209F
:100EC000694600900871487188711120FFF76FFA28
:100ED00069460D20FFF76BFA69461320FFF767FAA2
:100EE00069461420FFF763FA69461520FFF75FFA99
:100EF00069461620FFF75BFA69461720FFF757FA95
:100F000069460120FFF753FA69462A20FFF74FFA96
:100F10001CBD0000012203211046FFF75BFCFFF718
:100F2000F1FCFFF7E3F9FFF743FE114908690122DD
:100F30001043086100F0ACFAFFF78EFF0D4800F097
:100F400001FB00F029FA0020FFF75EFF012000F00E
:100F5000E3F809A0FFF746FE0E4C00F0BFF800F0E2
:100F6000FDF820680228F8D1FFF78EFFF5E70000B2
:100F700000E000E04C000020496E697469616C6912
:100F80007A6174696F6E20636F6D706C65746564EF
:100F90000D0A00006C000020254A10B50121904286
:100FA0000BD1437A002B08D1037C002B05D1C368F9
:100FB000962B02D301741FA036E090420FD1427AE3
:100FC000022A0CD1027C002A09D1C268962A06D8CE
:100FD00001741CA0FFF706FE00F04CF910BD144A86
:100FE0001C32904211D1427A012A0ED1027C002A91
:100FF0000BD1C268962A08D8017418A0FFF7F2FD39
:101000001C48006800F0ECF810BD094A38329042E4
:10101000FAD1427A012AF7D1027C002AF4D1C268BF
:10102000962AF1D8017414A0FFF7DCFD10BD000072
:10103000140000206B657930207A6B735F6B6565F7
:10104000700D0A006B657930207A6B735F66616C96
:101050006C696E675F656467650D0A006B65793161
:10106000207A6B735F726973696E675F6564676529
:101070000D0A0000700000206B657932207A6B73D6
:101080005F726973696E675F656467650D0A00006A
:1010900010B501210C4A04460846116000F03CF8E6
:1010A000002C08D0012C08D0022C08D0032C01D130
:1010B000FFF78EFE10BD002002E0012000E00220BC
:1010C000FFF7A2FE10BD00006C000020012110B54A
:1010D00041402A20FFF768FB10BD000010B50C4B03
:1010E000586800F02FF87D21C90088420CD90948C2
:1010F000006858601878002807D000201870002871
:1011000000D00120FFF7E2FF10BD0120F6E700004C
:10111000000000208400002010B501460120FFF7E8
:1011200043FB10BD10B51E20FFF782F9012800D047
:10113000002010BD10B51920FFF77AF9012800D062
:10114000002010BD0146044802680068401A8A4227
:1011500000D2401E704700008400002010B5064CED
:101160006068FFF7EFFF142805D9FFF76FFE606096
:10117000002000F0D1F910BD08000020012110B5B9
:1011800041401120FFF710FB10BD012110B5414077
:101190000D20FFF709FB10BD012110B541401320C0
:1011A000FFF702FB10BD012110B541401420FFF7ED
:1011B000FBFA10BD012110B541401720FFF7F4FAEA
:1011C00010BD012110B541401620FFF7EDFA10BD0A
:1011D000012110B541401520FFF7E6FA10BD0000CF
:1011E00070B501001D481C4C1D4D006812D001292E
:1011F0001BD0022924D003290BD1E16800F09EF80E
:101200000020686017A02168FFF7ECFC0320FFF7BF
:101210003FFF70BD216800F091F80120686011A0C7
:101220002168FFF7DFFC0020F1E7616800F086F835
:10123000022068600BA06168FFF7D4FC0120E6E79C
:10124000A16800F07BF80320686006A0A168FFF7A2
:10125000C9FC0220DBE700005C00002058000020F1
:101260006C00002070776D20675F647574793A2593
:101270006400000070B5224C2068002801D1FFF7FF
:10128000AFFFFFF7E3FD02252560A0600120FFF717
:1012900043FFE06801260300FFF7B4FC05040C14CB
:1012A0001D282700174918A02161FFF79BFC00208B
:1012B000E66018E01A4914A02161FFF793FC0120B1
:1012C000E56010E0174910A02161FFF78BFC0320B7
:1012D000E060022007E014490BA02161FFF782FCC7
:1012E0000420E060032000F0A3F870BD0FA026608A
:1012F000FFF778FC042000F09BF80020E06070BD50
:101300006C00002000DD6D00675F6F7A6F6E655FB7
:10131000776F726B5F74696D653A25640000000039
:101320000044950800E6DF0C00882A11636C6F7397
:10133000652074696D696E670000000070B50B4C24
:1013400005460E462046FFF70FFB00F025F8B1B228
:101350002046FFF77EFB0648008881B22046FFF753
:101360007EFBA9B22046FFF780FB70BD0020004045
:10137000580000201CB500206A46107050700221F1
:101380009170D070107101215171907169461220D5
:10139000FFF70DF81CBD00007FB5002468460472FD
:1013A000447284720321C1721F4E012502A9304686
:1013B0000395FFF7ACFA6846047045708470C470FA
:1013C00004714471857169463046FFF7FBFA0021CC
:1013D0003046FFF7D3FA02213046FFF7E1FA022147
:1013E0003046FFF7D4FA01213046FFF7E2FA002138
:1013F0003046FFF720FB0D48008881B23046FFF7EA
:1014000028FB0A4C241F208881B23046FFF727FBB7
:10141000208881B23046FFF728FBFFF7ABFF30464C
:10142000FFF7A7FA7FBD0000002000405C0000200D
:1014300010B50300FFF7E6FB050406111926250089
:10144000012020E00020FFF799FE0120FFF79DFE1C
:101450000020FFF7A1FE002011E00020FFF78EFE24
:101460000020FFF792FE0120F3E70020FFF786FE41
:101470000020FFF78AFE0020FFF78EFE0120FFF715
:1014800092FE10BD0020FFF779FE0020DEE700008D
:1014900070B586B0002468464470012505718570DA
:1014A000C47084714471047069462520FEF77FFF83
:1014B0006846457005718570C4708471447104700C
:1014C00069462420FEF773FFE1204002049068463D
:1014D0000575C47204730472447284720D4C02A9BF
:1014E0002046FFF7E7FA0122160431462046FFF7AF
:1014F000D8FA00212046FFF753FB0122114617209E
:10150000FFF7ACF920682843206020683043206052
:1015100006B070BD0060004070B5094D2878002805
:101520000CD0002406E001681C206043081800F07D
:101530002FF8641CA8684168A142F4DC70BD00006B
:1015400008000020F8B5114FB86001203870002461
:1015500017E01C2325465D432B4602680021093312
:10156000D15400682E1D80598047B968321D0B6820
:101570009854086880598047B96811350968641C17
:101580004855B8684168A142E3DCF8BD0800002076
:1015900010B50446C068401CE060606880477D224A
:1015A0006169D200914201D2491C6161217E814270
:1015B00002D00021616103E06169002900D06074FC
:1015C0002076617C204600F001F810BD70B50D4614
:1015D0000446017A0F4800268068A94211D0002DE8
:1015E00007D0E66026740121617282682046904728
:1015F00005E002216172826820469047E66025720C
:1016000070BD31466672002DFAD082682046904740
:1016100070BD00000800002074696D65726B65790B
:101620000000000067656172736B6579000000005F
:1016300050160000000000208C0000001E0C00006E
:10164000DC1600008C000020040400002E0C0000BA
:101650000100000000000000000000000000000089
:101660000000000018160000351100000000000006
:10167000000000000000000000000000000000006A
:1016800024160000251100000000000000000000EA
:101690000000000000000000000000001400002016
:1016A00002000000990F000080BB00000000000055
:1016B000E02E0000C05D00007FBB000000000000C5
:1016C0000100000000000000000000000000000019
:0C16D000006CDC020000000000000000C4
:04000005000000C136
:00000001FF
